:020000040000FA
:10000000830101308A007929FA00030E8301FB0085
:100010000A08FC008A010B1183160313BF0F112875
:10002000C00A83120317ED0F1628EE0A7C088A0017
:100030007B0E8300FA0E7A0E09001030F900F701EA
:10004000F801F60CF50C031C2B287408F80773084C
:10005000F7070318F80A0310F30DF40DF90B212824
:1000600008007508760403195628F701F8010130D5
:10007000F900F61B4028F90A0310F50DF60D392892
:1000800076087402031D462875087302031C4F2866
:100090007608F4027508F302031CF4030314F70D49
:1000A000F80DF60CF50CF90B40280800FF30F700AE
:1000B000F80008008B138B1B5A2874088A007308F9
:1000C00082000430831603139F0005149F13C13070
:1000D00083129F000A30F300F30B6C281F151F19C1
:1000E0006F281E080317C1000630831603139F00F4
:1000F000C730850008008312031306122821F30B72
:100100007E280608F0390338860086168728882856
:100110008612F3162821F30B8A2886168F2890283A
:1001200086122821861694289528861228210610E2
:1001300086169A289B2886122821283014210C30F4
:1001400014210630142183120313061201301421E6
:10015000F3162821F30BA92828298312031306126A
:1001600040307418F307F31715298312031306168A
:10017000C5208B17FF3903190800F30001308A00EE
:100180001521F60FB828F70AB8288B1377088A00CC
:10019000760882001030F3002730F400EF20FD08CD
:1001A000031DD3282D21E830F3000330F400EF20A5
:1001B000FD08031DDC282D216430F300F401EF203D
:1001C000FD08031DE4282D210A30F300F401EF207F
:1001D000FD08031DEC282D21303076071129FD087C
:1001E000031DFD03F801F80A7308F6027408031CE6
:1001F000740FF7020318F3287408F7077308F6075B
:100200000318F70A7803031D7E1408000F39F30062
:100210003030F3073A307302031C10290730F3071C
:100220007308831203130616F300F501730E0F39DA
:10023000F400831203130608F0397404860086164E
:10024000212922298612751A28297516730817295B
:100250004030F500F50B2A290800031DFD03F300CB
:10026000031D7E1430307E18F30720307E1CF30708
:10027000730811290008831203178C0083160C15CC
:100280008B138B1B402955308D00AA308D008C14A8
:100290008B178C1849290C1183128D0A840AF30BD1
:1002A0003A290800831603170C1483120C088000E7
:1002B0008D0A840AF30B52290800831603178C1346
:1002C00083128F0100308D0083130930F30020303A
:1002D00084003A2108000030831203178D008F013B
:1002E00083168C1383130930F300203084005221CD
:1002F000080020308B00831203130030850000308B
:100300008600003087008F308316810006309F0002
:10031000C7308500C0308600FF30870007309C0062
:100320008313203084008001840A841F932984165B
:100330008001840AF0300402031D982983171030CD
:1003400084008001840A70300402031DA1299030CA
:1003500084008001840AF0300402031DA9290430BE
:1003600083120313D100C4308316C4004030C80088
:100370004030D3007F30D500FF30DB00FF30E0009D
:10038000FF30E500FF30EA00403083120317BB0066
:100390007B206B218312031381010B118B176120CA
:1003A000831203132108003EAB002008023EAA007E
:1003B0000318AB0A00302D180138AC00F3012C08EB
:1003C000031DE7292008A0002108A100F129F30A54
:1003D0002C087302031DF1292A08A0002B08A10094
:1003E000F129831203134E1CFA292E18FA292E1410
:1003F0002D14002A831203132D104E18002A2E10DC
:1004000083120317B91F082A0313A001A1011B2A95
:10041000831203135D1F1B2A2F181B2A2F145D1B29
:10042000152AA00F1B2AA10A1B2A83120313A0035B
:10043000200F1B2AA103831203135D1B202A2F10F8
:10044000831203132108003EB1002008143EB000BF
:100450000318B10AF3013208031D332A2008A00053
:100460002108A1003D2AF30A32087302031D3D2A28
:100470003008A0003108A1003D2A00308312031388
:10048000AD180138B2002D1D4A2A33184A2A3314F8
:10049000AD14502A83120313AD102D19502A3310B6
:1004A000831203132108003EB5002008C83EB400A3
:1004B0000318B50AF3013608031D632A2008A000BB
:1004C0002108A1006D2AF30A36087302031D6D2A64
:1004D0003408A0003508A1006D2A003083120313F0
:1004E000AD190138B6002D1E7A2A37187A2A37142A
:1004F000AD15802A83120313AD112D1A802A3710EF
:100500000030831203132102B90002302002B80028
:10051000031CB9030030AD1B0138BA00F3013A08DF
:10052000031D972A2008A0002108A100A12AF30A90
:100530003A087302031DA12A3808A0003908A10057
:10054000A12A83120313CE1CAA2A3B18AA2A3B1401
:10055000AD17B02A83120313AD13CE18B02A3B1087
:100560000030831203132102BD0014302002BC00AE
:10057000031CBD03F3013E08031DC32A2008A0008D
:100580002108A100CD2AF30A3E087302031DCD2ADB
:100590003C08A0003D08A100CD2A003083120313BF
:1005A0003F180138BE00AD1EDA2A4018DA2A40147E
:1005B0003F14E02A831203133F10AD1AE02A4010C3
:1005C0000030831203132102C200C8302002C10090
:1005D000031CC203F3014308031DF32A2008A000F3
:1005E0002108A100FD2AF30A43087302031DFD2A16
:1005F0004108A0004208A100FD2A00308312031325
:10060000BF180138C3002D1F0A2B44180A2B4414AD
:10061000BF14102B83120313BF102D1B102B44107B
:10062000831203134B08F3004C08F4000030F5006C
:100630000130F60000308A00312003308A0077084C
:10064000C5007808C6000030F3000130F40045080A
:10065000F5004608F60000308A001D2003308A00AD
:100660007708C7007808C80048084C02CA00470845
:100670004B02C900031CCA032108013ECC0020081C
:10068000903ECB000318CC0AED1C492BA301A4011A
:100690005C2B831203136D1C5C2B4D185C2B4D14CB
:1006A000D71B562BA30F5C2BA40A5C2B83120313BE
:1006B000A303230F5C2BA403831203136D18612B78
:1006C0004D10831203134E1D6B2B4E1F6B2BCE1F31
:1006D0006B2B4E146E2B831203134E104E1D762B74
:1006E000CE1E762BCE1F762B2D15792B831203135E
:1006F0002D11CE1D812B4E1F812BCE1F812BCE1491
:10070000842B83120313CE10CE1D8C2BCE1E8C2B6C
:10071000CE1F8C2BAD168F2B83120313AD124E1DE3
:10072000972B4E1E972BCE1F972B2D169A2B83128D
:1007300003132D12CE1DA22B4E1EA22BCE1FA22BB9
:100740002D17A52B831203132D133F1DAB2BBF1D9C
:10075000AB2B4E15AE2B831203134E11BF1EB42BC1
:100760003F1EB42BCE15B72B83120313CE11BF1E21
:10077000BE2B4F18BE2B4F143F15C42B83120313EF
:100780003F11BF1AC42B4F1083120313BF1DCD2B73
:100790005018CD2B50143F16D32B831203133F1246
:1007A000BF19D32B501083120313871CD92BBF11F1
:1007B000DC2B83120313BF15071CE02BBF12E32BA6
:1007C00083120313BF164E19E92BCE19E92B3F13E1
:1007D000EC2B831203133F17071DF02B5113F32B40
:1007E0008312031351170317E91EF92B0313D201C8
:1007F000072C83120313BF1F072C5318072C531405
:10080000571A042CD20A072C83120313D203831223
:100810000313BF1B0C2C5310AC30F3001630F40044
:10082000831203135208F3070318F40A00308A00F6
:100830005A2083120313D4008B178A110A125418FA
:10084000232C5512242C5516D418282CD512292CBB
:10085000D51654192D2C55132E2C5517D419322C6E
:10086000D612332CD61657123F1F3E2C0317B91C35
:100870003E2CD4183E2C03135817412C831203131B
:1008800058133F1F472C561C472CD8144A2C831250
:100890000313D8103F1F502C581C502C5815532CA4
:1008A000831203135811D81E572CA501652C8312EF
:1008B0000313581F652C5918652C5914CE19622C36
:1008C000A50A652C83120313A50383120313581B77
:1008D0006A2C5910AC30F3001630F4008312031365
:1008E0002508F3070318F40A00308A005A208312FF
:1008F0000313DA008B178A110A125A18812C581226
:10090000822C5816DA18862CD811872CD8155A192B
:100910008B2C4E138C2C4E17DA19902CCE12912C56
:10092000CE165A1A952C4E12962C4E1604302502CD
:1009300083120313031CA02C0319A02CD816A12C7E
:10094000D812D81FA62CA601A701B92C8312031315
:10095000D81CB92C5B18B92C5B14CE19B32CA60F7C
:10096000B92CA70AB92C83120313A603260FB92C9E
:10097000A70383120313D818BE2C5B100330831215
:1009800003132702031DC62CE9302602831203132A
:10099000031DCC2CD817CD2CD81300305D1801388E
:1009A000DC00F3015C08031DDA2C2608A6002708EA
:1009B000A700E42CF30A5C087302031DE42CE83062
:1009C000A6000330A700E42CFF3083120313270294
:1009D000031DEC2CFF30260283120313031DF22C9F
:1009E0005D14F32C5D10DD1CF72CA801052D83127E
:1009F0000313581D052D5E18052D5E14DD1A022DFA
:100A0000A80A052D83120313A80383120313581990
:100A10000A2D5E10AC30F3001630F400831203137D
:100A20002808F3070318F40A00308A005A208312BA
:100A30000313DF008B178A110A125F18212D5D1135
:100A4000222D5D15DF18262DDD11272DDD155F19EF
:100A50002B2D5D122C2D5D160330280283120313FB
:100A6000031D342DDD14352DDD10DD125D1321083D
:100A7000003EE1002008013EE0000318E10A0030DA
:100A8000E31A0138E200F3016208031D4C2D20082F
:100A9000A0002108A100562DF30A62087302031D6D
:100AA000562D6008A0006108A100562D8312031383
:100AB000DD1F5F2D64185F2D64146316652D83128E
:100AC00003136312DD1B652D6410003083120313C2
:100AD0002102E60001302002E500031CE60300309D
:100AE00057180138E700F3016708031D7C2D200823
:100AF000A0002108A100862DF30A67087302031DD8
:100B0000862D6508A0006608A100862D83120313B8
:100B1000631C8F2D68188F2D6814D714952D8312A0
:100B20000313D7106318952D6810831203134E1DFD
:100B30009F2DD81D9F2DCE1F9F2DDD17A22D831217
:100B40000313DD13CE1DAA2DD81DAA2DCE1FAA2D4D
:100B50006314AD2D831203136310E31CB42D6918C5
:100B6000B42D6914D716BA2D83120313D712E318C4
:100B7000BA2D691083120313631DC32D6A18C32D88
:100B80006A145717C92D8312031357136319C92DFC
:100B90006A10831203134E1DD32D581ED32DCE1F62
:100BA000D32DE314D62D83120313E310CE1DDE2DB7
:100BB000581EDE2DCE1FDE2D6315E12D831203138B
:100BC0006311E31DE82D6B18E82D6B14D715EE2D7E
:100BD00083120313D711E319EE2D6B10003083122B
:100BE00003132402031DF62D043023028312031382
:100BF000031DFC2DE315FD2DE311631B032E631A6A
:100C0000032EE312062E83120313E316F3016C087E
:100C1000031D0F2E2308A3002408A400192EF30A95
:100C20006C087302031D192E0330A3000030A400CA
:100C3000192E0030831203136D1A0138EC00E31FE4
:100C4000262E6E18262E6E146D152C2E831203136D
:100C50006D11E31B2C2E6E10FF3083120313240240
:100C6000031D342EFF30230283120313031D3A2E7B
:100C7000E3173B2EE3135719412ED718412E571077
:100C8000442E831203135714E31D4B2E6F184B2E63
:100C90006F146317512E831203136313E319512E3C
:100CA0006F1083120313E31F5A2E70185A2E7014FC
:100CB0005715602E831203135711E31B602E70101B
:100CC000831203134908F3004A08F4000230F500C8
:100CD0000030F60000308A00312006308A007708A4
:100CE000F1007808F200003046028316A1000730B8
:100CF000831245028316A000031CA1032008F30001
:100D00002108F4008030F5000030F60000308A0041
:100D10001D2006308A007708A2007808A300720818
:100D20002307A50071082207A4000318A50A0330B1
:100D30003507A700E8303407A6000318A70AF30117
:100D400083122808031DAA2E83162608A800270848
:100D5000A900C22EF30A831228087302031DB62EBF
:100D600083162A08A8002B08A900C22EF30A8312B2
:100D700028087302031DC22E83162C08A8002D0814
:100D8000A900C22E83120313270883162702AB0083
:100D90008312260883162602AA00031CAB03270829
:100DA000831227078316AD002608831226078316B1
:100DB000AC000318AD0A2808F3002908F4000A3033
:100DC000F5000030F60000308A00312006308A003D
:100DD0007708AE007808AF000A30F3000030F40066
:100DE0002E08F5002F08F60000308A001D2006307E
:100DF0008A007708B0007808B10031082902B300F2
:100E000030082802B200031CB30300302502B500ED
:100E100068302402B400031CB5038312D71A142FC0
:100E2000571B142F6D10172F831203136D14571BAC
:100E30001B2FD7131E2F83120313D717F30183160B
:100E40003808031D282F3D08B6003E08B700332F91
:100E5000F30A831638087302031D332F3908B600CE
:100E60003A08B700332F00308312031351190138A9
:100E70008316B8003E08013EBA003D08F43EB900B2
:100E80000318BA0A83126D1D4C2F83163B184C2F82
:100E90003B148312ED15532F83120313ED116D19BB
:100EA000532F83163B1083120313ED1D5E2F831601
:100EB0003C185E2F3C1483126D16652F83120313AA
:100EC0006D12ED19652F83163C107D30F300003054
:100ED000F400831203132308F5002408F600003001
:100EE0008A001D2007308A0077088316BD00780825
:100EF000BE0000304002031D7F2F08303F02031C5C
:100F00008C2F0030C0020830BF02031CC003411BFD
:100F10008B2F41178C2F411383120313ED1F932F37
:100F20008316C201A32F83160313C11FAA2F4318D0
:100F3000AA2F43148312ED1AA02F8316C20AA32FDF
:100F400083160313C20383160313421CA92F4411F3
:100F5000AA2F441583160313C11BAF2F43102D3046
:100F600083160313420283120313031DB92F6D1757
:100F7000BA2F6D13ED126D1FC42F83164518C42FA1
:100F800045148312ED17CB2F83120313ED136D1B42
:100F9000CB2F8316451083160313441FD52FC41F70
:100FA000D52FC81FD52F4617D82F831603134613E6
:100FB0005B1CE02F481FE02F4E1CE02F4714E32F4F
:100FC000831603134710DB1CEB2F5B1DEB2FCE1C8E
:100FD000EB2FC714EE2F83160313C710DB1DF62F5C
:100FE0005B1EF62F4E1DF62F4715F92F83160313A0
:100FF00047118A15002800000000000000000000D2
:10100000DB1E08285B1F0828CE1D0828C7150B28E3
:1010100083160313C711DB1F1328601C13284E1EF1
:10102000132847161628831603134712601D1E281F
:10103000E01C1E28CE1E1E28C71621288316031367
:10104000C712E01D2928601E29284E1F292847178E
:101050002C28831603134713E01E3428601F3428FE
:10106000CD1C3428C717372883160313C713E01F76
:101070003F28651C3F28CE1F3F2846144228831670
:1010800003134610E51C4A28651D4A28491C4A28B6
:10109000C6144D2883160313C610E51D5528651E7A
:1010A00055284D1C552846155828831603134611FC
:1010B000E51E6028651F6028C91C6028C6156328C6
:1010C00083160313C611E51F6B286A1C6B28491D84
:1010D0006B2846166E28831603134612EA1C7628E0
:1010E0006A1D7628C91D7628C6167928831603132B
:1010F000C612EA1D81286A1E8128491E81284815CA
:101100008428831603134811EA1E8C286A1F8C2832
:10111000C91E8C28C8148F2883160313C810EA1F11
:101120009728551C9728491F972848149A288316F2
:1011300003134810D51CA228551DA228C91FA22898
:10114000C815A52883160313C811D51DAD28551E33
:10115000AD28411CAD284816B02883160313481249
:10116000D51EB828551FB828C11CB828C816BB28DA
:1011700083160313C812461BDE284718DE28C7183B
:10118000DE284719DE28C719DE28471ADE28C71AC5
:10119000DE28471BDE28C71BDE284618DE28C618B7
:1011A000DE284619DE28C619DE28461ADE28C61AA9
:1011B000DE28C61BDE2883120512E12883120313E2
:1011C000051683164819F028C818F0284818F02882
:1011D000C819F028481AF028C81AF028C613F328AE
:1011E00083160313C6174A18F728C813F828C81718
:1011F000831203171418002983160313C913032934
:1012000083160313C9178312031794180B29831627
:10121000031349130E298316031349174B18122978
:10122000411013294114CB181729C1101829C114D2
:10123000AC30F3001730F4005108F3070318F40A38
:1012400000308A005A2083160313CA008B178A15B0
:101250000A12B430F3001730F4005108F3070318F2
:10126000F40A00308A005A2083160313CB008B1730
:101270008A150A124F183E29CC113F29CC15CF18D8
:1012800043294911442949154F194829C9104929A9
:10129000C914CF194D294D104E294D144F1A5229FA
:1012A000491053294914CF1A5729CE135829CE175C
:1012B0004F1B5C29CD105D29CD14CF1B61294E1326
:1012C00062294E17F3015108031D6B290030CF002E
:1012D0000030D000A329F30A51087302031D7529B9
:1012E0000B30CF000030D000A329F30A510873025D
:1012F000031D872983120317640883160313CF0085
:1013000083120317650883160313D000A329F30A79
:1013100051087302031D9529831249088316CF00D3
:1013200083124A088316D000A329F30A51087302D6
:10133000031DA329831249088316CF0083124A088C
:101340008316D000A32983160313C11EA929D10136
:10135000B72983160313411EB7295218B72952140F
:101360004119B429D10AB72983160313D10383166F
:101370000313411ABC29521083160313411183121F
:10138000ED1FC7298316C11DC7294116CA29831617
:10139000031341120330510283160313031CD22995
:1013A000031DD429C115D529C111C112531BDC2934
:1013B000411FDF295314DF298316031353108316AB
:1013C0000313531CE729411FE729C117EA29831694
:1013D0000313C113531EEE295313F129831603136C
:1013E00053178312ED1BF9298316531DFC29D314BF
:1013F000FC2983160313D31083160313D318042A6E
:10140000C119042A5312072A831603135316D31D36
:101410000E2A54180E2A54145315142A8316031333
:101420005311D319142A5410003083160313510298
:1014300083160313031C202A0319202AD316212AFA
:10144000D312C41D2B2AD31E2B2AD31F2B2A441C94
:101450002B2AC4142E2A83160313C4102A304202E6
:1014600083160313031C362A031D382AD317392A7F
:10147000D3130130420283160313031C412A441480
:10148000422A44102C30420283160313031D4A2AB9
:10149000D5174B2AD513C41C532A5618532A561451
:1014A000831285165A2A8312031385128316C418D1
:1014B0005A2A561083160313441D632A5718632AA9
:1014C0005714C415692A83160313C4114419692AD1
:1014D000571083160313D51F722A5818722A5814EE
:1014E0004416782A831603134412D51B782A581001
:1014F00083160313441E802AD31E802AC416832A0F
:1015000083160313C4124417C4174208D9000230CB
:101510005902031C912A0319912A44130230D9005D
:10152000982A013059020318982AC4130130D900AF
:101530005B1448174208DA0004305A02031CA62A3A
:101540000319A62A5B100430DA00AD2A03305A02D0
:101550000318AD2A48130330DA00DB145B15420888
:10156000DC0006305C02031CBB2A0319BB2ADB101B
:101570000630DC00C22A05305C020318C22A5B1167
:101580000530DC00DB155B164208DD0008305D022B
:10159000031CD02A0319D02ADB110830DD00D72A1A
:1015A00007305D020318D72A5B120730DD00DB1617
:1015B0005B174208DE000A305E02031CE52A0319AD
:1015C000E52ADB120A30DE00EC2A09305E0203183D
:1015D000EC2A5B130930DE00DB1760144208DF00E1
:1015E0000C305F02031CFA2A0319FA2ADB130C30B1
:1015F000DF00012B0B305F020318012B60100B3052
:10160000DF006015E0144208E1000E306102031CA7
:101610000F2B03190F2B60110E30E100162B0D302C
:1016200061020318162BE0100D30E100E015601682
:101630004208E20010306202031C242B0319242B01
:10164000E0111030E2002B2B0F30620203182B2B1D
:1016500060120F30E200E01660174208E30012301B
:101660006302031C392B0319392BE0121230E300FB
:10167000402B113063020318402B60131130E3003C
:10168000E01765144208E40014306402031C4E2B7A
:1016900003194E2BE0131430E400552B1330640271
:1016A0000318552B65101330E400E5146515420846
:1016B000E60016306602031C632B0319632BE5104A
:1016C0001630E6006A2B1530660203186A2B651186
:1016D0001530E600E51565164208E7001830670288
:1016E000031C782B0319782BE5111830E7007F2BAA
:1016F0001730670203187F2B65121730E700E516D5
:1017000065174208E8001A306802031C8D2B031984
:101710008D2BE5121A30E800942B1930680203185B
:10172000942B65131930E800E5176A144208E900A4
:101730001C306902031CA22B0319A22BE5131C30D9
:10174000E900A92B1B3069020318A92B6A101B3072
:10175000E900EA146A154208EB001E306B02031C14
:10176000B72B0319B72BEA101E30EB00BE2B1D3030
:101770006B020318BE2B6A111D30EB00EA156A16C6
:101780004208EC0020306C02031CCC2B0319CC2B3C
:10179000EA112030EC00D32B1F306C020318D32B3E
:1017A0006A121F30EC00EA166A174208ED00223078
:1017B0006D02031CE12B0319E12BEA122230ED002C
:1017C000E82B21306D020318E82B6A132130ED005D
:1017D000EA1755144208EE0024306E02031CF62B63
:1017E0000319F62BEA132430EE00FD2B23306E0292
:1017F0000318FD2B55102330EE00D5145515420863
:10180000EF0026306F02031C0B2C03190B2CD51094
:101810002630EF00122C25306F020318122C5511C0
:101820002530EF00D5155516420883120317900096
:1018300028301002031C262C0319262C83160313B0
:10184000D5112830831203179000312C2730100255
:101850000318312C831603135512273083120317F4
:10186000900083160313D5165517420883120317E9
:1018700091002A301102031C472C0319472C8316B0
:101880000313D5122A30831203179100522C2930EA
:1018900011020318522C8316031355132930831297
:1018A0000317910083160313C41A592C8312851150
:1018B0005C2C83120313851503171218632C8316EF
:1018C0000313CE12662C83160313CE16831203174E
:1018D00092186E2C831603134E12712C8316031369
:1018E0004E16831203171219792C83160313CE1187
:1018F0007C2C83160313CE15831203179219842CA4
:10190000831603134E11872C831603134E1583126F
:101910000317121A8F2C83160313CE10922C8316E2
:101920000313CE1483120317921A9A2C83160313EF
:101930004E109D2C831603134E1483120317121B93
:10194000A52C831603134C11A82C831603134C15D6
:1019500083120317921BB02C83160313CC10B32CE5
:1019600083160313CC14F3015108031DBE2C003061
:1019700083120317920000309300F22CF30A5108EF
:101980007302031DCA2C003083120317920000302B
:101990009300F22CF30A51087302031DD62C831214
:1019A00003176008920061089300F22CF30A5108B3
:1019B0007302031DE42C83124508031792000313DE
:1019C000460803179300F22CF30A51087302031D13
:1019D000F22C8312450803179200031346080317DD
:1019E0009300F22C02308316031351028312031367
:1019F000031CFE2C0319FE2CD116FF2CD112F3016F
:101A000003171808031D092D1608940017089500E0
:101A1000182DF30A031718087302031D182D03135A
:101A20002308031794000313240803179500182DA7
:101A3000BC30F3001730F400831603130310510D6C
:101A4000F3070318F40A00308A005A2083120317A0
:101A50009600F30A0319F40A00308A005A20831210
:101A6000031797008B178A150A1200300313D11A37
:101A70000138031798001918512D831603134D1DB3
:101A8000512D0030F3000030F40000308A00AD200A
:101A9000CC30F6001730F70000308A00B5208A15E8
:101AA0000A12831603134D1D592D8312031719149F
:101AB0005C2D8312031719101A18722D8316031345
:101AC000CD1D722D0030F3000030F40000308A008C
:101AD000AD20DD30F6001730F70000308A00B52069
:101AE0008A150A1283160313CD1D7A2D831203174C
:101AF0001A147D2D831203171A1003135D1D852DF3
:101B000083164D1E852D4D15882D831603134D11FB
:101B100083125D19902D83164D1E902DCD15932D9A
:101B200083160313CD11831203171B18B02D8316D0
:101B300003134D1EB02D0030F3000130F4000030CF
:101B40008A00AD20831603132E08F6002F08F70035
:101B50007E100230FD0000308A00CA208A150A1269
:101B6000831603134D1EB82D831203171B14BB2DB0
:101B7000831203171B101C18D12D831603134D1E3F
:101B8000D12D0430F3000130F40000308A00AD2084
:101B9000EE30F6001730F70000308A00B5208A15C5
:101BA0000A12831603134D1ED92D831203171C141A
:101BB000DC2D831203171C101D18F72D8316031339
:101BC0004D1EF72D0530F3000130F40000308A007F
:101BD000AD20831603133208F6003308F7007E1099
:101BE0000530FD0000308A00CA208A150A128316CB
:101BF00003134D1EFF2D831203171D14022E831293
:101C000003171D101E181D2E831603134D1E1D2EA7
:101C10000630F3000130F40000308A00AD20831656
:101C200003133608F6003708F7007E140330FD0072
:101C300000308A00CA208A150A12831603134D1E2B
:101C4000252E831203171E14282E831203171E102D
:101C50001F183E2E831603134D1E3E2E0930F3002F
:101C60000130F40000308A00AD20F030F60017306B
:101C7000F70000308A00B5208A150A128316031374
:101C80004D1E462E831203171F14492E831203176D
:101C90001F1020185D2E261D5D2E0030F300003031
:101CA000F40000308A00AD20F430F6001730F70061
:101CB00000308A00B5208A150A1283120317261DE8
:101CC000632E2014662E83120317201021187A2EFB
:101CD000A61C7A2E0030F3000130F40000308A0098
:101CE000AD200530F6001830F70000308A00B5202E
:101CF0008A150A1283120317A61C802E2114832E24
:101D00008312031721102218972E261C972E0030BD
:101D1000F3000130F40000308A00AD201630F600E8
:101D20001830F70000308A00B5208A150A12831295
:101D30000317261C9D2E2214A02E83120317221097
:101D40002318B62E83160313CD1FB62E0030F300D2
:101D50000130F40000308A00AD202730F600183042
:101D6000F70000308A00B5208A150A128316031383
:101D7000CD1FBE2E831203172314C12E8312031707
:101D800023102418D72E831603134D1FD72E00308F
:101D9000F3000130F40000308A00AD203830F60046
:101DA0001830F70000308A00B5208A150A12831611
:101DB00003134D1FDF2E831203172414E22E831208
:101DC000031724102518F82E83160313CD1EF82EA2
:101DD0000030F3000130F40000308A00AD204930BB
:101DE000F6001830F70000308A00B5208A150A1274
:101DF00083160313CD1E002F831203172514032F00
:101E00008312031725100313581E0B2F0317261DCB
:101E10000B2FA6140E2F83120317A6100313D81D21
:101E2000162F0317261D162F2614192F831203179A
:101E3000261003134E1F232F0317261D232F83164F
:101E40000313CD17262F83160313CD138312CE1E33
:101E5000302F0317261D302F831603134D17332FF2
:101E6000831603134D1383124E1E3D2F0317261D99
:101E70003D2F83160313CD16402F83160313CD1267
:101E8000831203172718562FA61F562F0030F30072
:101E90000030F40000308A00AD205A30F6001830CF
:101EA000F70000308A00B5208A150A128312031742
:101EB000A61F5C2F27145F2F8312031727102818E3
:101EC000782FA61F782F0030F3000130F400003087
:101ED0008A00AD20831203172C08F6002D08F700A6
:101EE0007E100330FD0000308A00CA208A150A12D5
:101EF00083120317A61F7E2F2814812F8312031726
:101F000028102918952FA61F952F0330F3000130B4
:101F1000F40000308A00AD206B30F6001830F70076
:101F200000308A00B5208A150A1283120317A61FF3
:101F30009B2F29149E2F8312031729102A18B72FBD
:101F4000A61FB72F0430F3000130F40000308A00E0
:101F5000AD20831203173008F6003108F7007E1019
:101F60000530FD0000308A00CA208A150A1283124B
:101F70000317A61FBD2F2A14C02F831203172A1080
:101F80002B18D42FA61FD42F0530F3000130F400F6
:101F900000308A00AD206D30F6001830F7000030B8
:101FA0008A00B5208A150A1283120317A61FDA2F9A
:101FB0002B14DD2F831203172B1003132608F300B5
:101FC0002708F4000A30F5000030F60000308A00DF
:101FD00031200F308A0077080317AC007808AD0075
:101FE0008A110A160028000000000000000000000E
:101FF00000000000000000000000000000000000E1
:102000002C08F3002D08F4000A30F5000030F6002B
:1020100000308A001D2010308A007708AE00780852
:10202000AF002F08031327020317B1002E08031374
:1020300026020317B000031CB10332183128A61D75
:1020400031280030F3000030F40000308A00AD2069
:102050007930F6001830F70000308A00B5208A1178
:102060000A1683120317A61D372832143A28831242
:102070000317321033184E28261E4E280030F30066
:102080000130F40000308A00AD208A30F6001830AC
:10209000F70000308A00B5208A110A168312031750
:1020A000261E54283314572883120317331034186C
:1020B0006B28A61E6B280030F3000130F4000030BE
:1020C0008A00AD209B30F6001830F70000308A00FF
:1020D000B5208A110A1683120317A61E712834141C
:1020E000742883120317341035188828261F88286F
:1020F0000030F3000130F40000308A00AD20AC3035
:10210000F6001830F70000308A00B5208A110A1650
:1021100083120317261F8E28351491288312031764
:10212000351003135D1D99280317A61D992826163F
:102130009C288312031726120313DD1DA4280317FE
:10214000A61DA428A616A72883120317A6120313F8
:102150005D1EAF280317A61DAF282617B2288312CD
:10216000031726130313561DBA28D61DBA28831643
:102170004D16BD28831603134D128312D61CC52895
:10218000D61DC52803172615C82883120317261144
:102190000313561CD028D61DD0280317A617D32802
:1021A00083120317A6130313581CDB28D61DDB2844
:1021B0000317A615DE2883120317A6110313561E54
:1021C000E4280317B601EB288312031737180E29EA
:1021D000BA1E0E29B60A361CEF283817F028381315
:1021E000B61CF428B816F528B812361DF92839158A
:1021F000FA283911B61DFE28B915FF28B911361E67
:1022000003293A1704293A13B61E08293916092951
:102210003912361F0D293B150E293B118312031766
:10222000BA1E1429371417298312031737103C18C4
:102230002C290313561F2C290C30F3000130F40015
:1022400000308A00AD20BD30F6001830F7000030B5
:102250008A00B5208A110A1683120313561F3329E8
:1022600003173C143629831203173C103D184B29E1
:102270000313D61F4B290C30F3000130F40000305B
:102280008A00AD20C230F6001830F70000308A0016
:10229000B5208A110A1683120313D61F5229031779
:1022A0003D145529831203173D10831603134D1E49
:1022B000602983120317391C6029031356176329F9
:1022C00083120313561383164D1E6D2983120317B1
:1022D00039186D290313D617702983120313D613E7
:1022E000051D75290317391078298312031739142E
:1022F0000313CE1F80293F1F80298316D3158329FE
:1023000083160313D31183120317B9189229831666
:102310000313531F922983120317D418922903130E
:10232000CE17952983120313CE13D9302102031D32
:102330009B293030200283120317031CA3290319A1
:10234000A329B916A429B912D93003132102031DF8
:10235000AB29F9302002831203170318B12939176A
:10236000B2293913B91EB829391FB8293814BB2925
:10237000831203173810B81CC2293E18C2293E1414
:10238000B917C82983120317B913B818C8293E1002
:10239000FF30831203132102031DD029363020029F
:1023A00083120317031CD8290319D8293815D929F2
:1023B00038113818DF293819DF29B810E2298312BB
:1023C0000317B814381EE9293F18E9293F14B81536
:1023D000EF2983120317B811381AEF293F1083121F
:1023E0000317B819F8290313D719F829ED10FB2999
:1023F00083120313ED140317381D032A4018032A10
:1024000040143816092A8312031738123819092A7A
:1024100040109630831203174102831203170318EA
:10242000132AB817142AB8133B1C1B2A42181B2A5C
:102430004214BB15212A83120317BB113B18212A12
:10244000421083120317BB18292AB81F2C2A3B14E9
:102450002C2A831203173B1083120317BB1D392A42
:1024600003132918392A291401308A005D211230FA
:102470008A0083120317BB193F2A0313291003177D
:102480003B1A462A3B1F492ABB16492A83120317C7
:10249000BB1283120317BA1B512A3B1D542A3B1649
:1024A000542A831203173B12831203173B17BB1ED8
:1024B0005D2AB91D5D2ABB17602A83120317BB135F
:1024C000BB1F682A4318682A43140313D6156F2AC2
:1024D00083120313D6110317BB1B6F2A43108312F9
:1024E0000317BB1C762AC401C5018B2A831603136C
:1024F000411FCE2A831203174618CE2A4614C71846
:10250000852AC40F8B2AC50A8B2A83120317C4039A
:10251000440F8B2AC50383120317441C912A4714C6
:10252000922A4710C41C962A3A16972A3A12441D3A
:102530009B2ABA159C2ABA11C41DA02A3A15A12AB1
:102540003A11441EA52ABA14A62ABA10C41EAA2AF1
:102550003A14AB2A3A10441FAF2AC717B02AC71340
:10256000C41FB42A4717B52A4713451CB92AC716F2
:10257000BA2AC712C51CBE2A4716BF2A4712451DD4
:10258000C32AC715C42AC711C51DC82A4715C92A99
:102590004711451ECD2ABB14CE2ABB108316031348
:1025A000411BD52A83120317461083120317C71045
:1025B0003B1AE22A83160313411FE22A83120317F0
:1025C000BA16E52A83120317BA1203135118EF2A19
:1025D000D118EF2AD119EF2A0317BA13F22A83125E
:1025E0000317BA17391CFA2A4818FA2A4814031391
:1025F0005114012B83120313511003173918012BA7
:1026000048108312031739180B2B49180B2B491448
:102610000313D114122B83120313D1100317391C87
:10262000122B4910831203132108003E0317CB001D
:1026300003132008013E0317CA000318CB0A031333
:102640002008F3002108F4000230F5000030F60005
:1026500000308A00312013308A0077080317CC003D
:102660007808CD004A08F3004B08F4000230F5006A
:102670000030F60000308A00312013308A007708DD
:10268000CE007808CF004D084F02031D492B4C089F
:102690004E0283120313031D4F2B5111502B511562
:1026A000511E592B03175018592B50140313D115D1
:1026B000602B83120313D111511A602B0317501092
:1026C000831203173B19692BBA1B692B031356128C
:1026D0006C2B831203135616511B722B0317D10157
:1026E000D201872B83160313411FBB2B83120317C1
:1026F0005318BB2B5314D51A812BD10F872BD20A19
:10270000872B83120317D103510F872BD203831218
:102710000317511C8D2BD4158E2BD411D11C922B49
:102720005416932B5412511D972BD416982BD41258
:10273000D11D9C2B54179D2B5413511EA12BD41724
:10274000A22BD413D11EA62B5514A72B5510511F05
:10275000AB2BD514AC2BD510D11FB02B5515B12BED
:102760005511521CB52BD515B62BD511D21CBA2B31
:102770005516BB2B551283160313411BC22B831214
:102780000317531083120317D41CCB2B0313511FB1
:10279000CB2BBF17CE2B83120313BF13D11BD52B0B
:1027A0000317541CD82BD414D82B83120317D4101E
:1027B00083120317D41CE12B541DE12B0313D117F3
:1027C000E42B83120313D1130317541DEB2BD418DE
:1027D000EB2B5414EE2B831203175410551EF52BBC
:1027E0005618F52B56145415FB2B8312031754114E
:1027F000551AFB2B561083120317D512551B042CA8
:10280000D51F072CB914072C83120317B910831294
:102810000317B91C112C0313551D112C0317551741
:10282000142C8312031755130313551D1C2C031767
:10283000B9181C2CD5171F2C83120317D51303139B
:102840003F1B302C5518302CD518302C0317E91BA2
:10285000302C831603134C18302C83125112332C56
:10286000831203135116511B3C2C031757183C2C91
:10287000571403135514432C831203135510511F7F
:10288000432C0317571083120313511F4E2C0317A9
:1028900058184E2C58140313D514552C83120313B7
:1028A000D510511B552C0317581083120313511FB9
:1028B0005F2C0317D4185F2C0313D515622C8312D9
:1028C0000313D511D51D6B2C031759186B2C5914F4
:1028D00003135515722C831203135511D519722C3D
:1028E0000317591083120317B9187B2CD4187B2CAB
:1028F000031356157E2C8312031356110317B91CAC
:10290000862CD418862C0313D614892C8312031317
:10291000D6100317D41C912C0313551F912C581457
:10292000942C8312031358100317D41C9C2C0313EC
:10293000D51E9C2C56149F2C83120313561003177C
:10294000D41CA72C0313551EA72CD517AA2C831211
:102950000313D5130317691CB22C0313A201031729
:10296000DA01C82C83120317E91CC82C5B18C82C89
:102970005B14E919C12C0313A20FC82C0317DA0A40
:10298000C82C83120313A203220FC82C0317DA03E7
:1029900083120317E918CD2C5B108312031322084E
:1029A000F30003175A08F4005030F5000030F60029
:1029B00000308A001D2014308A007708DC00780877
:1029C000DD005D08013EDF005C08903EDE0003187C
:1029D000DF0A6708F3006808F4000030F5000130F2
:1029E000F60000308A00312014308A007708E000B9
:1029F0007808E1000030F3000130F4006008F500D1
:102A00006108F60000308A001D2015308A00770822
:102A1000E2007808E30063086802E50062086702E4
:102A2000E400031CE50303132208053E0317E60038
:102A30005E08F3005F08F4001030F5000030F60087
:102A400000308A00312015308A007708E7007808C6
:102A5000E80003133F1F352DD51F352D8316531F57
:102A6000352D83120317E914382D83120317E9104B
:102A7000F3016B08031D452D831603135108D10084
:102A8000831203176A08EA00532DF30A6B087302D6
:102A9000031D532D023083160313D100003083121F
:102AA0000317EA00532D0030831203176919013808
:102AB000EB00E91C602D6C18602D6C146915662DF7
:102AC000831203176911E918662D6C10831203171E
:102AD000EF18742D6F18802D0313CE1D802D031752
:102AE000ED01EE01EF14E9150030831203176E02B9
:102AF000031D7C2D10306D02031C802DEF10E91199
:102B000083120313CE1D872D03176F148A2D831292
:102B100003176F1023300313220283120317031CC1
:102B2000952D0319952D6914962D6910691A9E2DFE
:102B30000313D61A9E2D0317E912A12D8312031732
:102B4000E916D41CAA2D83161018AA2D101483126E
:102B50006916B12D831203176912D418B12D83168B
:102B60001010831603171118C82D8312691FC82D62
:102B70000030F3000030F40000308A00AD20C73090
:102B8000F6001830F70000308A00B5208A110A16C6
:102B900083120317691FCF2D83161114D22D8316AC
:102BA000031711101218EB2D8312691FEB2D003043
:102BB000F3000130F40000308A00AD2083120317C7
:102BC0006608F600F7017E100230FD0000308A0032
:102BD000DC208A110A1683120317691FF22D83164F
:102BE0001214F52D83160317121013180A2E8312D0
:102BF000691F0A2E0230F3000130F40000308A0011
:102C0000AD20D830F6001830F70000308A00B5202B
:102C10008A110A1683120317691F112E83161314C3
:102C2000142E83160317131083120313D51F1D2EA2
:102C3000D61D1D2E03176917202E83120317691343
:102C4000D418292E83161418292E14148312E91768
:102C5000302E83120317E913D41C302E8316141060
:102C600083120317D41C3B2E831615183B2E151404
:102C700003134C14442E831603134C1083120317B2
:102C8000D418442E831615108316031717184A2ECE
:102C900096104B2E96149718502E03134912522E4D
:102CA00003134916E730F3001830F4005108F30716
:102CB0000318F40A00308A005A208316031797007D
:102CC0008B178A110A160313CC1D6C2E0317161CC2
:102CD0006C2E03134C166F2E831603134C12CC1D4F
:102CE000772E03171618772E03134C177A2E831698
:102CF00003134C135108023C83160317031D822E45
:102D00001614832E1610961C8A2E16188A2E03135C
:102D1000CC168D2E83160313CC120317961C952EFA
:102D2000161C952E0313CC17982E83160313CC1361
:102D3000CC1B9E2E4C1B9E2EC912A12E8316031354
:102D4000C9164C1AA72ECC1AA72EC911AA2E831663
:102D50000313C9150A12CF2901340234043408348C
:102D60001034203440348034083409340A340B34AD
:102D70000C340D340E340F34103411341234133437
:102D80001434153416341734183419341A341B34E7
:102D90001C341D341E341F34203421342234233497
:102DA0002434253426342734283429342A342B3447
:102DB0002C342D342E342F343034313432343334F7
:102DC0003434353436343734383439343A343B34A7
:102DD0003C343D343E343F34403441344234433457
:102DE0004434453446344734483449344A344B3407
:102DF0004C344D344E344F345034513452345334B7
:102E00005434553456345734583459345A345B3466
:102E10005C345D345E345F34603461346234633416
:102E20006434653466346734683469346A346B34C6
:102E30006C346D346E346F34703471347234733476
:102E40007434753476347734783479347A347B3426
:102E50007C347D347E347F348034813482348334D6
:102E60008434853486348734883489348A348B3486
:102E70008C348D348E348F34903491349234933436
:102E80009434953496349734983499349A349B34E6
:102E90009C349D349E349F34A034A134A234A33496
:102EA000A434A534A634A734A834A934AA34AB3446
:102EB000AC34AD34AE34AF34B034B134B234B334F6
:102EC000B434B534B634B734B834B934BA34BB34A6
:102ED000BC34BD34BE34BF34C034C134C234C33456
:102EE000C434C534C634C734C834C934CA34CB3406
:102EF000CC34CD34CE34CF34D034D134D234D334B6
:102F0000D434D534D634D734D834D934DA34DB3465
:102F1000DC34DD34DE34DF34E034E134E234E33415
:102F2000E434E534E634E734E834E934EA34EB34C5
:102F3000EC34ED34EE34EF34F034F134F234F33475
:102F4000F434F534F634F734F834F934FA34FB3425
:102F5000FC34FD34FE34FF340034003401340134D9
:102F6000013461346134613400340134003402349A
:102F700002340234023402340034003400340034A9
:102F80000034003400340034043400340534003498
:102F90000634003407340034563443344F3420347C
:102FA0006634723465346B34763465346E3463342D
:102FB0006934613420342034003456346534743438
:102FC00065346C3420346634723465346B34763452
:102FD00065346E3463346934613400342E34003423
:102FE0004D3448347A3400344634723465346B34AA
:102FF000763465346E3463346934613420346C342F
:1030000065347034653473340034313432342C34E4
:1030100035346B3448347A3420342034203420342E
:103020002034203420342034203400342034203420
:10303000353430346B3448347A34203420342034FE
:103040002034203420342034203420340034203400
:103050003134303430346B3448347A3420342034D2
:1030600020342034203420342034203420340034E0
:1030700020342034203431344D3448347A342034F0
:1030800020342034203420342034203420342034A0
:10309000003420342034313430344D3448347A34E0
:1030A0002034203420342034203420342034203480
:1030B000203400344B344634203466347234653462
:1030C0006B34763465346E3463346934613420345F
:1030D0002034203400342E3400344D3448347A34D3
:1030E0002034203420342034203420342034203440
:1030F00000344634723465346B3476342E342034E4
:103100006B3469346A3465346C347A3465347334BE
:1031100020340034563443344F34203420342034A7
:1031200020342034203420342034203420342034FF
:10313000203420340034563443344F342D344B344F
:1031400046342034203420342034203420342034B9
:103150002034203420340034563443344F342B345C
:103160004B3446342034203420342034203420346E
:10317000203420342034203400344C346F34633411
:103180006B34003420342034203420340034523462
:10319000653466346534723465346E34633469344E
:1031A000613420344F3453344334203420340034D9
:1031B0004D3448347A3420342034203420342034C0
:1031C000203420342034203420342034003400349F
:0E31D00001340034003404340534063407346E
:084000000000010000000000B7
:02400E003A3F37
:1042000000000000000000000000000000000000AE
:10421000000000000000000000000000000000009E
:10422000000000000000000000000000000000008E
:10423000000000000000000000000000000000007E
:10424000000000000000000000000000000000006E
:10425000000000000000000000000000000000005E
:10426000000000000000000000000000000000004E
:10427000000000000000000000000000000000003E
:10428000000000000000000000000000000000002E
:10429000000000000000000000000000000000001E
:1042A000000000000000000000000000000000000E
:1042B00000000000000000000000000000000000FE
:1042C00000000000000000000000000000000000EE
:1042D00000000000000000000000000000000000DE
:1042E00000000000000000000000000000000000CE
:1042F00000000000000000000000000000000000BE
:1043000000000000000000000000000000000000AD
:10431000000000000000000000000000000000009D
:10432000000000000000000000000000000000008D
:10433000000000000000000000000000000000007D
:10434000000000000000000000000000000000006D
:10435000000000000000000000000000000000005D
:10436000000000000000000000000000000000004D
:10437000000000000000000000000000000000003D
:10438000000000000000000000000000000000002D
:10439000000000000000000000000000000000001D
:1043A000000000000000000000000000000000000D
:1043B00000000000000000000000000000000000FD
:1043C00000000000000000000000000000000000ED
:1043D00000000000000000000000000000000000DD
:1043E00000000000000000000000000000000000CD
:1043F00000000000000000000000000000000000BD
:00000001FF
